:030000000200AE4D
:03008B000257E237
:2000AE001266DD1265770258140820413334345F3820077657616C7465720876773234304F
:2000CE00373030D20C22200C030200DED2AED2BE227401908128F0A37400F0908124E0FC84
:2000EE00A3E0FDECFAEDFB908128E0D39AA3E064806303809B400302014BC004C00512000A
:20010E00D4D005D0047401908126F0A37400F0908126E0D3941EA3E0648094804003020154
:20012E003D908126E004F07004A3E004F080E0908128E004F07004A3E004F0809E22740171
:20014E0090812AF0A37400F090812AE0D39402A3E064809480400302017690812AE004F095
:20016E007004A3E004F080E022904002E0548070F82290812CE060030201C9120177743872
:20018E00904000F01201777438904000F01201777438904000F0120177740C904000F012C9
:2001AE0001777402904000F01201777406904000F01201777401904000F022200D030201AB
:2001CE00D02290812CE0D3941050030201F01201777401904000F090812CE0C394109081F1
:2001EE002CF090812CE0D39408500302020990812CE0243790812CF002021490812CE0C34C
:20020E00940190812CF012017790812CE04480904000F07401908137F090812DE0FE908109
:20022E0037E0D39E4003020259120177908137E090812D2582F58250020583E0904001F0FF
:20024E00908137E004F0600380CF0022908138E090812CF09081397C2D7D8175070A750658
:20026E00001264B3120180908143E0FAA3E0FBEA908124F0A3EBF01200DF741190812CF0D8
:20028E008001009002907C2D7D8175070A7506001264D912018022740190812CF090814509
:2002AE007C2D7D8175070A7506001264B31201807409908138F090814F7C397D8175070A7D
:2002CE007506001264B3908159E0FAA3E0FBEA908143F0A3EBF012025A22C20D740090811A
:2002EE002CF08001009002F27C2D7D8175070A7506001264D912018022C20E740090815B73
:20030E00F0740090815CF0746490815DF02230EC0302032B740190815FF002033174009058
:20032E00815FF030B30302034190815FE0440290815FF030B50302035190815FE044049057
:20034E00815FF090815FE090815EF02212031C90815EE0908161F0A20E740033FE90816145
:20036E00E024FFEE82E040030203BC7401908138F0800908204C6F636B6564209003817CB7
:20038E00397D8175070A7506001264D97464908143F0A37400F012025A7400908160F074EE
:2003AE000090815BF0740090815CF002045890815BE0FE908161E06E700302041690815D9D
:2003CE00E0FE90815CE0C39EE433FE90815BE0FA908161E0D39AB3EE72E040030204079096
:2003EE00815BE0FE7404FAEEC333DAFCFE908161E04E908160F002040D7400908160F074AE
:20040E000090815CF002045090815DE0FE90815CE0C39E400302043990815CE0240190811C
:20042E005CF07400908160F002045090815BE0FE7404FAEEC333DAFCFE908161E04E908112
:20044E0060F0908161E090815BF022908166E0FCA3E0FDECFAEDFB908162E0D39AA3E06426
:20046E00806303809B500302048B908166E0FAA3E0FBEA908168F0A3EBF00204CD908164A1
:20048E00E0FCA3E0FDECFAEDFB908162E0C39AA3E064806303809B40030204BD908164E031
:2004AE00FAA3E0FBEA908168F0A3EBF00204CD908162E0FAA3E0FBEA908168F0A3EBF02254
:2004CE007B00126268EA908170F0A3EBF07B001263B9908170E0FAA3E0FBEA908162F0A36C
:2004EE00EBF090816AE0FAA3E0FBEA908164F0A3EBF090816CE0FAA3E0FBEA908166F0A3AA
:20050E00EBF0120459908168E0FAA3E0FBEA90816EF0A3EBF0227B00125978908176125D65
:20052E00EC7B001263B9908176125DCA908172125DEC22C2F890817AE090817DF0A374009E
:20054E0000F07C087D0090817DE0FAA3E0FB12647890817BE0FC7D00EA4CFAEB4DFBEA9006
:20056E00817DF0A3EBF0740190817CF090817CE0D3941040030205BCD29590817DE05400FC
:20058E00FAA3E05480FBEA4B24FFB392947C017D0090817DE0FAA3E0FB126478EA90817D8A
:2005AE00F0A3EBF0C29590817CE004F080BED2F822740090817AF074FF90817BF0120541A7
:2005CE002275B1A0744190F700F0908180E0FEEE60030205EC747190F704F00205FAEE6493
:2005EE000160030205FD745390F704F002060BEE6402600302060E744990F704F002061C07
:20060E00EE6403600302061F744790F704F002062DEE64046003020630744390F704F0025D
:20062E00063EEE64056003020641744190F704F002064FEE64066003020652744090F7048A
:20064E00F0020652742590F705F0740790F701F0740090817FF07401908182F0908182E0DB
:20066E00D3940F400302072E908182E075F010A490F7002582F582500205837455F09081A7
:20068E0082E075F010A490F7002582F58250020583A37455F0908182E075F010A490F700E3
:2006AE002582F58250020583A3A3A3A3A3A37400F0908182E075F010A490F7002582F582CD
:2006CE0050020583A3A37400F0908182E075F010A490F7002582F58250020583A3A3A37420
:2006EE0000F0908182E075F010A490F7002582F58250020583A3A3A3A37400F0908182E08E
:20070E0075F010A490F7002582F58250020583A3A3A3A3A37400F0908182E004F002066AC7
:20072E00908181E0FE7401FAEEC333DAFC90F700F0908181E0540164016003020759E59A2B
:20074E00FEEE4402F59AD2AF020762E59AFE7402F45EF59A22200F03020774E59AFEEE448A
:20076E0002F59A02077DE59AFE7402F45EF59A227C037D00908183E0FAA3E0FB126485EA91
:20078E0090F706F07C057D00908183E0FAA3E0FB126478EA90F707F07C037D00908185E01C
:2007AE00FAA3E0FB126485EA90F70CF090F70DE0541F7C057D00FE908185E0FAA3E0FB1268
:2007CE006478EA4E90F70DF022908188125FC7125F4915000000125EF37401125F63EA908B
:2007EE00F708F0908188125FC7125F490D000000125EF37401125F63EA90F709F0908188B5
:20080E00125FC7125F4905000000125EF37401125F63EA90F70AF0908188125FC7125F4931
:20082E0003000000125F047401125F63EA54F890F70BF090818C125FC7125F49150000008D
:20084E00125EF37401125F63EA90F70CF090818C125FC7125F490D000000125EF3740112EB
:20086E005F63EA90F70DF090818C125FC7125F4905000000125EF37401125F63EA90F70E7B
:20088E00F090818C125FC7125F4903000000125F047401125F63EA54F890F70FF02290811B
:2008AE0092E0FEEE60030208D0908191E075F010A490F7002582F58250020583747FF00290
:2008CE000905EE64016003020908908191E075F010A490F7002582F58250020583A374FB07
:2008EE00F0908191E075F010A490F7002582F5825002058374BFF002093DEE6402600302BC
:20090E000940908191E075F010A490F7002582F58250020583A374D7F0908191E075F01091
:20092E00A490F7002582F5825002058374BFF0020975EE64036003020978908191E075F0C1
:20094E0010A490F7002582F58250020583A374E7F0908191E075F010A490F7002582F58228
:20096E005002058374BFF002097822908193E075F010A490F7002582F58250020583A3A365
:20098E00A3A3A3A3C082C083908193E075F010A490F7002582F58250020583A3A3A3A3A3ED
:2009AE00A3E054F74408D083D082F0908193E0908191F0908194E0908192F01208AC2290D4
:2009CE008195E075F010A490F7002582F58250020583A3A3A3A3A3A3C082C083908195E09E
:2009EE0075F010A490F7002582F58250020583A3A3A3A3A3A3E054F7D083D082F090819519
:200A0E00E0908191F0908196E0908192F01208AC22908197E075F010A490F7002582F5820E
:200A2E0050020583E05482FE908197E075F010A490F7002582F58250020583A3E0FA740108
:200A4E00FCEAC313DCFC54554EFE908197E075F010A490F7002582F58250020583A3A3A3F6
:200A6E00A3A3A3E054084EFE908197E075F010A490F7002582F58250020583A3A3A3A3A3A8
:200A8E00A3E0FA7403FCEAC333DCFC54204E908198F022908199E075F010A490F700258252
:200AAE00F58250020583A3A37C037D00C082C08390819AE0FAA3E0FB126485EAD083D08283
:200ACE00F0908199E075F010A490F7002582F58250020583A3A3A37C057D00C082C08390FA
:200AEE00819AE0FAA3E0FB126478EA54E0D083D082F0908199E075F010A490F7002582F50E
:200B0E008250020583A3A3A3A3A3A3C082C083908199E075F010A490F7002582F58250027A
:200B2E000583A3A3A3A3A3A3E054FBD083D082F02290819CE075F010A490F7002582F5821C
:200B4E0050020583A3A3C082C08390819D125FC7125F4915000000125EF37401125F63EA97
:200B6E00D083D082F090819CE075F010A490F7002582F58250020583A3A3A3C082C08390AF
:200B8E00819D125FC7125F490D000000125EF37401125F63EAD083D082F090819CE075F00D
:200BAE0010A490F7002582F58250020583A3A3A3A3C082C08390819D125FC7125F4905003E
:200BCE000000125EF37401125F63EAD083D082F090819CE075F010A490F7002582F5825041
:200BEE00020583A3A3A3A3A3C082C08390819D125FC7125F4903000000125F047401125FAB
:200C0E0063EA54F8D083D082F090819CE075F010A490F7002582F58250020583A3A3A3A3E7
:200C2E00A3A3C082C08390819CE075F010A490F7002582F58250020583A3A3A3A3A3A3E004
:200C4E0054FB4404D083D082F0229081A1E075F010A490F7002582F58250020583A3A3A325
:200C6E00A3A3A3E0540464046003020D549081A1E075F010A490F7002582F58250020583ED
:200C8E00A3A3E0FA7B00E4125F639081A6125FDD9081A6125FC7125F4908000000125F04C8
:200CAE009081A1E075F010A490F7002582F58250020583A3A3A3E0FA7B00E4125F63125E96
:200CCE00E59081A6125FDD9081A6125FC7125F4908000000125F049081A1E075F010A490BB
:200CEE00F7002582F58250020583A3A3A3A3E0FA7B00E4125F63125EE59081A6125FDD9074
:200D0E0081A6125FC7125F4905000000125F049081A1E075F010A490F7002582F582500290
:200D2E000583A3A3A3A3A3E0FE7403FAEEC313DAFC541FFA7B00E4125F63125EE59081A659
:200D4E00125FDD020DB99081A1E075F010A490F7002582F58250020583A3A3E0FA7B00E4C6
:200D6E00125F639081A6125FDD9081A6125FC7125F4903000000125F049081A1E075F01064
:200D8E00A490F7002582F58250020583A3A3A3E0FE7405FAEEC313DAFC5407FA7B00E41288
:200DAE005F63125EE59081A6125FDD9081A6125FC79081A2125FDD229081ABE0D39408509C
:200DCE0003020DD874089081ABF09081ABE0D394005003020E6A9081AAE075F010A490F7E8
:200DEE00002582F58250020583C082C08374009081AEF09081ABE0C39401FE9081AEE0D3E1
:200E0E009E4003020E66E58124FFF88682088683A3A3A3A3A3A3A3C082C0839081AEE0D06A
:200E2E0083D0822582F58250020583C082C0839081ACE0FCA3E0FD8C828D83E0D083D08296
:200E4E00F09081ACE004F07004A3E004F09081AEE004F06003809C00D083D0829081AAE0C6
:200E6E0075F010A490F7002582F58250020583A3A3A3A3A3A3C082C0839081AAE075F01065
:200E8E00A490F7002582F58250020583A3A3A3A3A3A3E0540FFE9081ABE0540FC44ED083AA
:200EAE00D082F090817FE06003020F0B90F701E0641824FFE433FE90F701E0641F24FFEEDB
:200ECE0072E04003020EE390F701E090817FF0740790F701F09081AAE075F010A490F70066
:200EEE002582F58250020583A3E0540264026003020F0B90817FE0442090817FF09081AA1F
:200F0E00E075F010A490F7002582F58250020583A374FEF0229081B0E0FCA3E0FD8C828D6C
:200F2E0083C082C0839081AFE075F010A490F7002582F58250020583A3A3A3A3A3A3E0C4ED
:200F4E00540FD083D082F09081B0E0FCA3E0FD8C828D83E0D394085003020F799081B0E083
:200F6E00FCA3E0FD8C828D837408F09081B0E0FCA3E0FD8C828D83E0D39400500302102551
:200F8E009081AFE075F010A490F7002582F58250020583C082C08374009081B4F09081B09C
:200FAE00E0FCA3E0FD8C828D83E0C39401FE9081B4E0D39E40030210219081B2E0FCA3E0C5
:200FCE00FD8C828D83C082C083E58124FDF88682088683C082C083D083D082A3A3A3A3A372
:200FEE00A3A3C082C0839081B4E0D083D0822582F58250020583E0D083D082F09081B2E0BE
:20100E0004F07004A3E004F09081B4E004F06003808B00D083D08290817FE0600302107FD3
:20102E0090F701E0641824FFE433FE90F701E0641F24FFEE72E0400302105790F701E09094
:20104E00817FF0740790F701F09081AFE075F010A490F7002582F58250020583A3E0540888
:20106E006408600302107F90817FE0442090817FF09081AFE075F010A490F7002582F58250
:20108E0050020583A374FDF0229081B5E0908197F0120A1F908198E0548064806003021013
:2010AE00C29081B5E0908197F0120A1F908198E0544170ED9081B5E0908191F074009081AF
:2010CE0092F01208AC9081B5E0908199F09081B6E0FAA3E0FBEA90819AF0A3EBF0120AA19B
:2010EE009081B5E09081AAF09081B8E09081ABF09081B9E0FAA3E0FBEA9081ACF0A3EBF005
:20110E00120DC69081B5E0908193F07403908194F012097922125D3A0000C842125D3A0084
:20112E00004842125DFD125C239081BBE075F002A49080112582F58250020583E0FAA3E0ED
:20114E00FB7401125AEF125CA19081BCE0FAA3E0FB7400125AEF125C23125ACE12646DEA1B
:20116E009081BEF0A3EBF022125D3A0000C842125D3A00004842125DFD125C239081C0E06E
:20118E0075F002A49080012582F58250020583E0FAA3E0FB7401125AEF125CA19081C1E044
:2011AE00FAA3E0FB7400125AEF125C23125ACE12646DEA9081C3F0A3EBF022125D3A000035
:2011CE00C842125D3A00008C42125DFD125C239081C5E075F002A49080112582F582500231
:2011EE000583E0FAA3E0FB7401125AEF125CA19081C5E075F002A490809F2582F582500242
:20120E000583E0FAA3E0FB7401125AEF125C23125D3A0000C842126121125D3A0000A041AE
:20122E00125DFD125C231261349081C5E075F002A49080012582F58250020583E0FAA3E0D5
:20124E00FB1261217401125AEF125CA11261349081C5E075F002A490808F2582F58250029B
:20126E000583E0FAA3E0FB1261217401125AEF125C23126134125BAF125ACE12646DEA9031
:20128E0081C6F0A3EBF0227C057D009081C8E0FAA3E0FB126485EA9081CAF0227C057D006A
:2012AE009081CBE0FAA3E0FB126478908023E0FCA3E0FDEA4CFAEB4DFBEA9081CDF0A3EBC6
:2012CE00F0229081D3E09081DBF09081D4E09081DCF09081D5E09081DDF09081D6E0908130
:2012EE00DEF09081D7E09081DFF09081D8E09081E0F09081D9E09081E1F09081DAE0908138
:20130E00E2F09081CFE09081B5F09081D0E0FAA3E0FBEA9081CBF0A3EBF01212AA9081CD5E
:20132E00E0FAA3E0FBEA9081B6F0A3EBF09081D2E09081B8F09081DBAA82AB83EA9081B9B2
:20134E00F0A3EBF0121097229081E3E09081B5F09081E4E0FAA3E0FBEA9081CBF0A3EBF02B
:20136E001212AA9081CDE0FAA3E0FBEA9081B6F0A3EBF09081E6E09081B8F09081E7AA8288
:20138E00AB83EA9081B9F0A3EBF0121097229081F0E0FCA3E0FD8C828D83E060030213CF72
:2013AE009081F0E0FCA3E0FD8C828D837401F09081F2E0FCA3E0FD8C828D837408F0021341
:2013CE00F19081F2E0FCA3E0FD8C828D83C082C0839081F0E0FCA3E0FD8C828D83E0D0835E
:2013EE00D082F02274F49081F0F0A37481F074F69081F2F0A37481F012139C9081F4E0907F
:20140E0081F5F09081F6E0FE9081F5E0D39E40030214A174019081CFF074219081D0F0A3D4
:20142E007400F074039081D2F09081F5E09081D3F09081F5E075F002A490807F2582F58298
:20144E0050020583E0FAA3E0FBEB9081D4F09081F5E075F002A490807F2582F58250020597
:20146E0083E09081D5F074009081D6F074009081D7F074009081D8F074009081D9F074007F
:20148E009081DAF01212D09081F5E004F06003021411002274F79081F0F0A37481F074F998
:2014AE009081F2F0A37481F012139C9081F7E09081F8F09081F9E0FE9081F8E0D39E40037C
:2014CE0002155174019081CFF074239081D0F0A37400F074039081D2F09081F8E09081D3CB
:2014EE00F09081F8E075F002A49080DF2582F58250020583E0FAA3E0FBEB9081D4F09081EA
:20150E00F8E075F002A49080DF2582F58250020583E09081D5F074009081D6F0740090816D
:20152E00D7F074009081D8F074009081D9F074009081DAF01212D09081F8E004F0600302B6
:20154E0014C1002274FA9081F0F0A37481F074FC9081F2F0A37481F012139C9081FAE09078
:20156E0081FBF09081FCE0FE9081FBE0D39E400302160174019081CFF074269081D0F0A3FA
:20158E007400F074039081D2F09081FBE09081D3F09081FBE075F002A49080FF2582F582AB
:2015AE0050020583E0FAA3E0FBEB9081D4F09081FBE075F002A49080FF2582F582500205B0
:2015CE0083E09081D5F074009081D6F074009081D7F074009081D8F074009081D9F074001E
:2015EE009081DAF01212D09081FBE004F06003021571002274FD9081F0F0A37481F074FFC4
:20160E009081F2F0A37481F012139C9081FDE09081FEF09081FFE0FE9081FEE0D39E400302
:20162E000216B174019081CFF074289081D0F0A37400F074039081D2F09081FEE09081D3FD
:20164E00F09081FEE075F002A49080CF2582F58250020583E0FAA3E0FBEB9081D4F0908192
:20166E00FEE075F002A49080CF2582F58250020583E09081D5F074009081D6F07400908116
:20168E00D7F074009081D8F074009081D9F074009081DAF01212D09081FEE004F06003024F
:2016AE001621002274009081F0F0A37482F074029081F2F0A37482F012139C908200E090A0
:2016CE008201F0908202E0FE908201E0D39E400302176174019081CFF0742A9081D0F0A31F
:2016EE007400F074039081D2F0908201E09081D3F0908201E075F002A49080AF2582F5828C
:20170E0050020583E0FAA3E0FBEB9081D4F0908201E075F002A49080AF2582F58250020597
:20172E0083E09081D5F074009081D6F074009081D7F074009081D8F074009081D9F07400BC
:20174E009081DAF01212D0908201E004F060030216D1002274039081F0F0A37482F07405ED
:20176E009081F2F0A37482F012139C908203E0908204F0908205E0FE908204E0D39E400384
:20178E0002181174019081CFF0742C9081D0F0A37400F074039081D2F0908204E09081D32F
:2017AE00F0908204E075F002A49080BF2582F58250020583E0FAA3E0FBEB9081D4F0908239
:2017CE0004E075F002A49080BF2582F58250020583E09081D5F074009081D6F074009081BF
:2017EE00D7F074009081D8F074009081D9F074009081DAF01212D0908204E004F0600302E7
:20180E001781002274069081F0F0A37482F074089081F2F0A37482F012139C908206E090CB
:20182E008207F0908208E0FE908207E0D39E40030218A574019081CFF0742F9081D0F0A361
:20184E007400F074029081D2F0908207E09081D3F0908207E09080782582F5825002058387
:20186E00E09081D4F074009081D5F074009081D6F074009081D7F074009081D8F074009073
:20188E0081D9F074009081DAF01212D0908207E004F06003808D002274099081F0F0A374A9
:2018AE0082F0740B9081F2F0A37482F012139C908209E090820AF090820BE0FE90820AE0EE
:2018CE00D39E400302193974019081CFF074089081D0F0A37400F074029081D2F090820AF4
:2018EE00E09081D3F090820AE09080702582F58250020583E09081D4F074009081D5F0743F
:20190E00009081D6F074009081D7F074009081D8F074009081D9F074009081DAF01212D0B8
:20192E0090820AE004F06003808D002290820DE0908210F090820CE0908211F0908210E0F3
:20194E00FAA3E0FBEA90820EF0A3EBF022908212E0D39408500302196D7408908212F07415
:20196E0001908229F0908212E0FE908229E0D39E40030219BF908229E090821F2582F58218
:20198E0050020583C082C083908213E0FCA3E0FD8C828D83E0D083D082F0908213E004F0CD
:2019AE007004A3E004F0908229E004F0600380B500908212E090821FF090821F7C157D82A1
:2019CE0075070A7506001264B32280080743414E2049443A9019DB7D007C017F077E0012D1
:2019EE0062D17E007F0590822AE0FAA3E0FB12632180040320443A901A027D007C017F032D
:201A0E007E001262D190822CE0D394005003021A63740190822FF090822CE0FE90822FE0BB
:201A2E00D39E4003021A6390822DE0FCA3E0FD8C828D837E007F04E0FA7B0012632B9082A4
:201A4E002DE004F07004A3E004F090822FE004F0600380C3007B001263B922908230E09054
:201A6E008234F0A3740000F07C087D00908234E0FAA3E0FB126478908231E0FC7D00EA4C4C
:201A8E00FAEB4DFBEA908232F0A3EBF022908236E09080782582F58250020583E0FE9082B5
:201AAE0037E0D39E5003021B1B908236E0C39401FC7401126492FE908030E04E908030F070
:201ACE007420FB7A01780290802D1264F86003021AF0743FFB7A01780290802D75070312E9
:201AEE0064A5908236E09080702582F58250020583C082C083908236E09080782582F582DC
:201B0E0050020583E0D083D082F0021B91908237E0C394324003021B75908236E0C39401B3
:201B2E00FC7401126492FE908030E04E908030F07420FB7A01780290802D1264F8600302EE
:201B4E001B60743FFB7A01780290802D7507031264A5908236E09080702582F58250020565
:201B6E00837432F0021B91908236E09080702582F58250020583C082C083908237E0D083EF
:201B8E00D082F0908236E0C39401FC740112649290817AF0908236E09080702582F582506B
:201BAE00020583E090817BF012054122C20F120763908239E0FEA3E0B40006BE0003021B26
:201BCE00D2021BE3908238E0908236F07432908237F0121A9B908238E075F002A490807F59
:201BEE002582F58250020583C082C083908239E0FAA3E0FBEA908162F0A3EBF074F0908177
:201C0E0064F0A374D8F07400908166F0A37400F0120459D083D082C082C083908168E0FAB5
:201C2E00A3E0FBEAD083D082F0A3EBF0D20F120763221205BF740190823BF090823BE0D314
:201C4E0094084003021C8490823BE09080782582F5825002058374F2F090823BE09082387B
:201C6E00F07400908239F0A37400F0121BBA90823BE004F080C52290823CE075F002A49078
:201C8E0080FF2582F58250020583C082C08390823DE0FAA3E0FBEAD083D082F0A3EBF09006
:201CAE00823CE075F002A490810F2582F582500205837400F0A37400F022740190823FF012
:201CCE0090823FE0D394084003021CF790823FE090823CF0740090823DF0A37400F0121CA7
:201CEE008590823FE004F080D722908240E0C39401FE7403FAEEC333DAFC908240F09082AC
:201D0E0040E0540864086003021D23908240E04440908240F0908240E05470448E90824016
:201D2E00F0D29512014CD2967401908245F0908245E0D394084003021D76908240E0548037
:201D4E0024FFB3929412014CC295908240E0FE7401FAEEC333DAFC908240F012014CD29562
:201D6E00908245E004F080C6D294908241E0FCA3E0FD8C828D837400F0A37400F0908243F1
:201D8E00E0FCA3E0FD8C828D837400F0A37400F03091FDC2957401908245F0908245E0D375
:201DAE00940C4003021E9212014CD295908241E0FCA3E0FD8C828D83C082C083908241E035
:201DCE00FCA3E0FD8C828D837C017D00E0FAA3E0FB126478EAD083D082F0A3EBF0908243C9
:201DEE00E0FCA3E0FD8C828D83C082C083908243E0FCA3E0FD8C828D837C017D00E0FAA390
:201E0E00E0FB126478EAD083D082F0A3EBF012014C209003021E53908241E0FCA3E0FD8C2E
:201E2E00828D83C082C083908241E0FCA3E0FD8C828D83E04401FAA3E04400FBEAD083D0C2
:201E4E0082F0A3EBF020F903021E87908243E0FCA3E0FD8C828D83C082C083908243E0FC3C
:201E6E00A3E0FD8C828D83E04401FAA3E04400FBEAD083D082F0A3EBF0C295908245E00446
:201E8E00F0021DA9C29622A210929722201103021F02D20974019081CFF074009081D0F049
:201EAE00A37400F074039081D2F0908028E09081D3F0A20974003354019081D4F090812327
:201ECE00E09081D5F074009081D6F074009081D7F074009081D8F074009081D9F074009008
:201EEE0081DAF01212D0D210121E957404908000F0021F0FC210121E95C209740090802838
:201F0E00F0227401908246F0908246E0D39408400302215C908246E075F002A49080EF2514
:201F2E0082F58250020583C082C083908246E075F002A49080DF2582F58250020583E0FA37
:201F4E00A3E0FBEAD083D082F0A3EBF0C20F120763908246E0908240F0908246E075F00292
:201F6E00A490808F2582F58250020583AA82AB83EA908241F0A3EBF0908246E075F002A4D0
:201F8E0090809F2582F58250020583AA82AB83EA908243F0A3EBF0121CF8908246E075F0C2
:201FAE0002A49080AF2582F58250020583C082C083908246E09081BBF0908246E075F0029E
:201FCE00A490809F2582F58250020583E0FAA3E0FBEA9081BCF0A3EBF0121123D083D08240
:201FEE00C082C0839081BEE0FAA3E0FBEAD083D082F0A3EBF0908246E075F002A49080BF18
:20200E002582F58250020583C082C083908246E09081C0F0908246E075F002A490808F2535
:20202E0082F58250020583E0FAA3E0FBEA9081C1F0A3EBF0121176D083D082C082C08390EA
:20204E0081C3E0FAA3E0FBEAD083D082F0A3EBF0908246E075F002A49080CF2582F5825049
:20206E00020583C082C083908246E09081C5F01211C9D083D082C082C0839081C6E0FAA3DB
:20208E00E0FBEAD083D082F0A3EBF0908246E075F002A49080DF2582F58250020583C082EE
:2020AE00C083908246E075F002A49080AF2582F58250020583C082C083908246E075F002B1
:2020CE00A49080BF2582F58250020583E0FCA3E0FDD083D082E0C39CFAA3E09DFBEAD083F5
:2020EE00D082F0A3EBF0D20F120763908246E09080302582F58250020583C082C0839082AE
:20210E0046E075F002A490808F2582F58250020583E0C394FFA3E06480948FE433FE908202
:20212E0046E075F002A490809F2582F58250020583E0C394FFA3E06480948FEE82E0E43392
:20214E00D083D082F0908246E004F0021F16227464908049F0A37400F0740A90804BF0A3C3
:20216E007400F074D490806DF0A374FEF0746490806FF0A37400F07401908247F0908247CE
:20218E00E0D3940840030221ED908247E075F002A49080372582F582500205837400F0A305
:2021AE007400F0908247E075F002A490804B2582F582500205837400F0A37400F090824752
:2021CE00E075F002A490805B2582F582500205837400F0A37400F0908247E004F0809E22CB
:2021EE00908248E0D3940850030222037401908027F0022220908248E0C3940140030222D5
:20220E00187408908027F0022220908248E0908027F0908027E0FA7B0090802A7F01E41214
:20222E0061472274499081F0F0A37482F0744B9081F2F0A37482F012139C908249E0908246
:20224E004AF090824BE0FE90824AE0D39E40030222E074019081CFF074039081D0F0A37463
:20226E0000F074039081D2F090824AE09081D3F090824AE075F002A49080372582F582500A
:20228E00020583E0FAA3E0FBEB9081D4F090824AE075F002A49080372582F5825002058308
:2022AE00E09081D5F074009081D6F074009081D7F074009081D8F074009081D9F074009024
:2022CE0081DAF01212D090824AE004F0600302225000223009030225AB740190824CF09027
:2022EE00824CE0D3940840030225AB90824CE075F002A490804B2582F58250020583E0D34F
:20230E009400A3E09400500302244690824CE09080302582F582500205837400F090824C0D
:20232E00E075F002A490804B2582F58250020583C082C08390824CE075F002A490804B2503
:20234E0082F58250020583E0C39401FAA3E09400FBEAD083D082F0A3EBF090824CE075F0B8
:20236E0002A490805B2582F58250020583E0D39400A3E0940050030223D8742AFB7A01780C
:20238E000290802D7507031264A590824CE075F002A490805B2582F58250020583C082C0A8
:2023AE008390824CE075F002A490805B2582F58250020583E0C39401FAA3E09400FBEAD0E2
:2023CE0083D082F0A3EBF002244390824CE075F002A49080DF2582F58250020583C082C011
:2023EE008390806DE0FCA3E0FDD083D082E0FAA3E0FBD31265155003022443C002C0039046
:20240E00824CE0908248F01221EED003D00290824CE075F002A490804B2582F582500205D7
:20242E00837400F0A37400F090824CE0908028F0D211121E9A0225A290824CE075F002A47B
:20244E009080DF2582F58250020583C082C08390824CE075F002A49080EF2582F58250024A
:20246E000583E0FCA3E0FDD083D082E0C39CFAA3E09DFB90806FE0FCA3E0FDAE02AF03EC48
:20248E00FAEDFBEED39AEF64806303809B50030225A290824CE075F002A49080372582F555
:2024AE008250020583E0FEA3E0B4FF06BEFF0302250EC004C005C20F120763D005D0049094
:2024CE00824CE075F002A49080372582F58250020583C082C08390824CE075F002A4908018
:2024EE00372582F58250020583E02401FAA3E03400FBEAD083D082F0A3EBF0D20F12076394
:20250E0090824CE0908249F0122231200A0302253090824CE0908248F01221EE740490800A
:20252E0000F090824CE09080302582F582500205837400F090824CE075F002A490804B25FA
:20254E0082F58250020583C082C083908049E0FAA3E0FBEAD083D082F0A3EBF090824CE029
:20256E0075F002A490805B2582F58250020583C082C08390804BE0FAA3E0FBEAD083D08218
:20258E00F0A3EBF0742AFB7A01780290802D7507031264A590824CE004F00222ED229081E4
:2025AE0022E060030227D3740190824DF090824DE0D3940840030227C890824DE090803087
:2025CE002582F58250020583E0FEA209B3EE82E040030227AE90824DE075F002A49080DF16
:2025EE002582F58250020583C082C08390824DE075F002A490810F2582F58250020583E00E
:20260E00FCA3E0FDD083D082E02CFAA3E03DFB90824DE075F002A490807F2582F582500281
:20262E000583E0FCA3E0FDAE02AF03ECFAEDFBEEC39AEF64806303809B40030226AB9082B1
:20264E004DE09080702582F58250020583E0D39400500302268EC004C00590824DE090829D
:20266E0036F090824DE09080702582F58250020583E0C39401908237F0121A9BD005D0048E
:20268E0090824DE075F002A490810F2582F582500205837400F0A37400F00227AB90824D2C
:2026AE00E075F002A49080DF2582F58250020583C082C08390824DE075F002A490810F2526
:2026CE0082F58250020583E0FCA3E0FDD083D082E0C39CFAA3E09DFB90824DE075F002A47A
:2026EE0090807F2582F58250020583E0FCA3E0FDAE02AF03ECFAEDFBEED39AEF6480630325
:20270E00809B500302277390824DE09080702582F58250020583E0C394FF4003022756C032
:20272E0004C00590824DE0908236F090824DE09080702582F58250020583E0240190823746
:20274E00F0121A9BD005D00490824DE075F002A490810F2582F582500205837400F0A3742E
:20276E0000F00227AB90824DE075F002A490810F2582F58250020583C082C08390824DE061
:20278E0075F002A49080FF2582F58250020583E0FAA3E0FBEAD083D082F0A3EBF00227BFDC
:2027AE0090824DE0908236F07400908237F0121A9B90824DE004F00225BB908121E09081E8
:2027CE0022F00227DE908122E0C39401908122F022200903022819908029E024019080293C
:2027EE00F0908029E0540464046003022819741190812CF08001009028047C2D7D8175074A
:20280E000A7506001264D912018022A20A740033FE7420FB7A01780290802D1264F824FF7E
:20282E00B3EE82E040030228477421FB7A01780290802D7507031264A5908000E0FEEE603B
:20284E0003022915908027E075F002A49080AF2582F58250020583E0FAA3E0FB90824E7F17
:20286E0005E4126147740190812CF01261EA90802D74011261667441FB7A017802E4126121
:20288E006690824E74011261667456FB7A017802E41261667C2D7D8175070A750600126481
:2028AE00B3120180908027E075F002A49080BF2582F58250020583E0FAA3E0FB90824E7FA4
:2028CE0005E4126147740990812CF01261EA90802A74011261667442FB7A017802E41261BB
:2028EE006690824E74011261667456FB7A017802E41261667C2D7D8175070A750600126421
:20290E00B31201800229D2EE640160030229D5908027E075F002A490807F2582F58250028F
:20292E000583E0FAA3E0FB90824E7F05E4126147740190812CF01261EA90802D7401126103
:20294E00667444FB7A017802E412616690824E74011261667456FB7A017802E41261667CFD
:20296E002D7D8175070A7506001264B3120180908027E075F002A49080DF2582F5825002E0
:20298E000583E0FAA3E0FB90824E7F06E4126147740990812CF01261EA90802A740112619D
:2029AE006690824E74011261667456FB7A017802E41261667C2D7D8175070A750600126460
:2029CE00B3120180022A65EE64026003022A68740190812CF01261EA90802D74011261663D
:2029EE0080080720496E707574209029F074021261667C2D7D8175070A7506001264B3120F
:202A0E000180908027E075F002A49080CF2582F58250020583E0FAA3E0FB90824E7F06E40D
:202A2E00126147740990812CF01261EA90802A740112616690824E74011261667456FB7A52
:202A4E00017802E41261667C2D7D8175070A7506001264B3120180022AE8EE6403600302FE
:202A6E002AEB740190812CF01261EA90802D740112616680080720204441432020902A8395
:202A8E0074021261667C2D7D8175070A7506001264B3120180908027E09080702582F582C0
:202AAE0050020583E0FA7B0090824E7F07E4126147740990812CF01261EA90802A7401128D
:202ACE00616690824E74011261667C2D7D8175070A7506001264B3120180022B71EE64041B
:202AEE006003022B74740190812CF01261EA90802D740112616680080720537061726B7317
:202B0E00902B0674021261667C2D7D8175070A7506001264B3120180908027E075F002A411
:202B2E009080372582F58250020583E0FAA3E0FB90824E7F077401126147740990812CF031
:202B4E001261EA90802A740112616690824E74011261667C2D7D8175070A7506001264B303
:202B6E00120180022B747420FB7A01780290802D7507031264A57400908030F02290825888
:202B8E00E0908000F0908000E0FEEE6003022BA1022BA9EE64016003022BB2740A90815DE3
:202BAE00F0022BCBEE64036003022BBD022BC5EE64046003022BCE741E90815DF0022BCEEC
:202BCE0022A212920A22908000E0FEEE64026003022C3112035A908160E0FEEE64106003CC
:202BEE00022BFD7401908258F0122B8B022C13EE64206003022C16908027E0C3940190822B
:202C0E0048F01221EE022C2BEE64406003022C2E908027E02401908248F01221EE022C2EA0
:202C2E00022D70EE64016003022D7312035A908160E0FEEE64106003022C557400908258AB
:202C4E00F0122B8B022C6BEE64206003022C6E908027E0C39401908248F01221EE022C8319
:202C6E00EE64406003022C86908027E02401908248F01221EE022CBDEE64336003022CC035
:202C8E00908027E0908238F0908027E075F002A490807F2582F58250020583E0240AFAA381
:202CAE00E03400FBEA908239F0A3EBF0121BBA022CF8EE64556003022CFB908027E09082EB
:202CCE0038F0908027E075F002A490807F2582F58250020583E0C3940AFAA3E09400FBEADE
:202CEE00908239F0A3EBF0121BBA022D32EE64316003022D35908027E0908238F0908027F3
:202D0E00E075F002A490807F2582F58250020583E02401FAA3E03400FBEA908239F0A3EBCF
:202D2E00F0121BBA022D6DEE64516003022D70908027E0908238F0908027E075F002A4906A
:202D4E00807F2582F58250020583E0C39401FAA3E09400FBEA908239F0A3EBF0121BBA029E
:202D6E002D70022DC6EE6003022DC912035A908160E0FEEE64106003022D95740390825842
:202D8E00F0122B8B022DABEE64206003022DAE908027E0C39401908248F01221EE022DC315
:202DAE00EE64406003022DC6908027E02401908248F01221EE022DC6022E1EEE6403600379
:202DCE00022E2112035A908160E0FEEE64106003022DED7404908258F0122B8B022E03EE3A
:202DEE0064206003022E06908027E0C39401908248F01221EE022E1BEE64406003022E1E40
:202E0E00908027E02401908248F01221EE022E1E022ED3EE64046003022ED612035A90816D
:202E2E0060E0FEEE64106003022E457402908258F0122B8B022E5BEE64206003022E5E90F6
:202E4E008027E0C39401908248F01221EE022E73EE64406003022E76908027E0240190828E
:202E6E0048F01221EE022E9EEE64036003022EA1908027E075F002A49080372582F58250BD
:202E8E000205837400F0A37400F0740090815CF0022EB7EE64056003022EBAA209B39211D2
:202EAE00121E9A740090815CF0022ED0EE64066003022ED3A20AB39212122BCF7400908117
:202ECE005CF0022ED3022ED622740090825FF090825EE0C39401FE90825FE0D39E400302EB
:202EEE002F4790825FE0FC7D007A007BF61263C7EAFCEBFD900000EC2582F582E5833DF55B
:202F0E0083C082C08390825FE0FC7D0090825CE02CFAA3E03DFBEAFCEBFD900000EC2582B1
:202F2E00F582E5833DF583E493D083D082F090825FE004F060038097007A007BF612657052
:202F4E002274AA905555F07455902AAAF07490905555F090825BE0FC7D00908259E02CFA77
:202F6E00A3E03DFBEAFCEBFD900000EC2582F582E5833DF583E090825BF074AA905555F07E
:202F8E007455902AAAF074F0905555F0908259E0FCA3E0FD900000EC2582F582E5833DF57D
:202FAE0083E0908259F0A3740000F02222908260E05400FAA3E05440FBEA908259F0A3EB75
:202FCE00F0908262E090825BF0902F4FAA82AB83EA90825CF0A3EBF0902FBAAA82AB8390B1
:202FEE002F4FAC02AD03AA82AB83ECC39AFAED9BFBEA90825EF0122ED790825BE0908263A4
:20300E00F02274AA905555F07455902AAAF074F0905555F0908259E0FCA3E0FD900000EC5A
:20302E002582F582E5833DF583E090825BF02222908264E0FAA3E0FBEA908259F0A3EBF035
:20304E00903010AA82AB83EA90825CF0A3EBF090303DAA82AB83903010AC02AD03AA82AB16
:20306E0083ECC39AFAED9BFBEA90825EF0122ED790825BE0908266F02274AA905555F07405
:20308E0055902AAAF074A0905555F0908259E0FCA3E0FD900000EC2582F582E5833DF583BD
:2030AE00C082C08390825BE0D083D082F0908259E0FCA3E0FD900000EC2582F582E5833D95
:2030CE00F583E05480FE90825BE054806E70DE22908267E0FAA3E0FBEA908259F0A3EBF025
:2030EE00908269E090825BF0903087AA82AB83EA90825CF0A3EBF09030DEAA82AB839030EB
:20310E0087AC02AD03AA82AB83ECC39AFAED9BFBEA90825EF0122ED72290826AE0FAA3E040
:20312E00FBEA908267F0A3EBF090826CE0908269F01230DE90826AE02401FAA3E03400FB9F
:20314E00EA908267F0A3EBF090826DE0908269F01230DE2290826EE0FAA3E0FBEA90825957
:20316E00F0A3EBF0908270E090825BF07A007BF61265702274AA905555F07455902AAAF0BB
:20318E007480905555F074AA905555F07455902AAAF0908259E0FCA3E0FD900000EC2582B4
:2031AE00F582E5833DF5837430F0908259E0FCA3E0FD900000EC2582F582E5833DF583E07B
:2031CE005480648070E422908271E05400FAA3E05440FBEA908259F0A3EBF0903182AA82BE
:2031EE00AB83EA90825CF0A3EBF09031D5AA82AB83903182AC02AD03AA82AB83ECC39AFA9F
:20320E00ED9BFBEA90825EF0122ED722908277E0D39400A3E0940050030232CF908275E0F6
:20322E00FAA3E0FBEA908267F0A3EBF0908273E0FCA3E0FD900000EC2582F582E5833DF522
:20324E0083E0908269F01230DE7401908279F0A37400F0908277E0C39401FAA3E09400FBAE
:20326E00908279E0D39AA3E09B40030232CF908279E0FCA3E0FD908275E02CFAA3E03DFBD5
:20328E00EA90826EF0A3EBF0908279E0FCA3E0FD908273E02CFAA3E03DFBEAFCEBFD9000BD
:2032AE0000EC2582F582E5833DF583E0908270F0123162908279E004F07004A3E004F08018
:2032CE00922290827FE0D39400A3E0940050030233637400908281F0A37400F090827FE0E3
:2032EE00C39401FAA3E09400FB908281E0D39AA3E09B4003023363908281E0FCA3E0FD9004
:20330E00827DE02CFAA3E03DFBEAFCEBFD900000EC2582F582E5833DF583C082C0839082C3
:20332E0081E0FCA3E0FD90827BE02CFAA3E03DFBEAFCEBFD900000EC2582F582E5833DF552
:20334E0083E0D083D082F0908281E004F07004A3E004F0808722908283E0FEEE60030233F3
:20336E0076C2B2C2B4023382EE64016003023385D2B2C2B4023391EE64026003023394C2B6
:20338E00B2D2B40233A0EE640360030233A3D2B2D2B40233A3227E007F01908001E0FAA3F2
:2033AE00E0FB12632B7420FA7C017D007E047F011262D17E007F01908023E0FAA3E0FB121A
:2033CE00632B7420FA7C017D007E047F011262D17E007F01908025E0FA7B0012632B7B00DF
:2033EE001263B97401908284F0908284E0D39408400302345C908284E075F002A49080113A
:20340E002582F582500205837E007F07E0FAA3E0FB12632B7420FA7C017D007E047F01120E
:20342E0062D1908284E075F002A49080012582F582500205837E007F07E0FAA3E0FB1263F0
:20344E002B7B001263B9908284E004F0809B22740190812CF0800908536176696E672E2EEC
:20346E009034657C2D7D8175070A7506001264D91201807401908283F01233647400908262
:20348E0071F0A37400F01231D5908001AA82AB83EA908273F0A3EBF07400908275F0A37454
:2034AE0000F0908026AA82AB83908001AC02AD03AA82AB83ECC39AFAED9BFBEA908277F08C
:2034CE00A3EBF012321A7400908283F012336480060553617665649034E07D007C017F05C0
:2034EE007E001262D17B001263B9227401908283F0123364740090827BF0A37400F0908085
:20350E0001AA82AB83EA90827DF0A3EBF0908026AA82AB83908001AC02AD03AA82AB83EC16
:20352E00C39AFAED9BFBEA90827FF0A3EBF01232D07400908283F0123364908001E0FEA372
:20354E00E0B4FF06BEFF0302355B0235C67400908001F0A37400F07400908023F0A374004B
:20356E00F07402908025F07401908285F0908285E0D3940840030235C3908285E075F002B5
:20358E00A49080012582F582500205837410F0A37427F0908285E075F002A4908011258284
:2035AE00F582500205837410F0A37427F0908285E004F080B812345D22908286E09082898F
:2035CE00F0908287E0FE908289E0D39E4003023652908289E09080782582F58250020583C2
:2035EE00C082C083908288E0908162F0A3740000F07432908164F0A37400F074F290816665
:20360E00F0A37400F0120459D083D082C082C083908168E0D083D082F0908289E09082365B
:20362E00F0908289E09080702582F58250020583E0908237F0121A9B908289E004F06003E7
:20364E000235CF00227420FA7C017D007E047F011262D17B001263B98035342D2D2D2D2DF2
:20366E002D2D2D2D2D2D2D2D2D2D2D2D2D2D2D2D2D2D2D2D2D2D2D2D2D2D2D2D2D2D2D2D9C
:20368E002D2D2D2D2D2D2D2D2D2D2D2D2D2D2D9036697D007C017F347E001262D17B00124D
:2036AE0063B980181747454D20566F6C746167652047656E657261746F723A201261EA9058
:2036CE0036B274021261669000B774021261669000C874021261667D007C01E0A3FF7E026C
:2036EE001262D17B001263B97423FA7C017D007E047F011262D17E007F01908001E0FAA370
:20370E00E0FB12632B7B001263B980050443414E3A90371B7D007C017F047E001262D17E42
:20372E00007F01908023E0FAA3E0FB12632B7420FA7C017D007E047F011262D17E007F0103
:20374E00908025E0FA7B0012632B7B001263B980171650687973696B2E496E73742E2C201D
:20376E00556E692048443A201261EA90375F74021261669000C074021261667D007C01E0BE
:20378E00A3FF7E021262D17B001263B98035342D2D2D2D2D2D2D2D2D2D2D2D2D2D2D2D2D25
:2037AE002D2D2D2D2D2D2D2D2D2D2D2D2D2D2D2D2D2D2D2D2D2D2D2D2D2D2D2D2D2D2D2D5B
:2037CE002D2D2D90379D7D007C017F347E001262D17B001263B9802B2A3F20202020202003
:2037EE002020202020202048656C7020286E206368616E6E656C3D312E2E382C20303D6187
:20380E006C6C299037E77D007C017F2A7E001262D17B001263B9801F1E21206E20202020F0
:20382E0020202020202020417474656E74696F6E204D6F64756C659038277D007C017F1ED8
:20384E007E001262D17B001263B9801C1B23206E20202020202020202020204D6F64756C25
:20386E00655F4E722053657490385B7D007C017F1B7E001262D17B001263B9803F3E262004
:20388E006E2C627228302E2E3629202043414E204944266261756472617465282832302C8E
:2038AE0035302C3130302C3132352C3235302C3530302C314D487A292053657490388C7DDE
:2038CE00007C017F3E7E001262D17B001263B9802A2941206E2C762F61206E202020202032
:2038EE00412043616C6962726174696F6E2F4120766F6C74616765204765749038E07D000A
:20390E007C017F297E001262D17B001263B9802A2942206E2C762F62206E202020202042C2
:20392E002043616C6962726174696F6E2F4220766F6C746167652047657490391F7D007C4D
:20394E00017F297E001262D17B001263B9801E1D43206E2F6320202020202020202043685B
:20396E00616E6E656C205365742F47657490395E7D007C017F1D7E001262D17B001263B967
:20398E008033324420702C746578743C63723E2020446973706C6179207465787420617430
:2039AE0020706F7374696F6E20702028303D756E6C6F636B299039917D007C017F327E0050
:2039CE001262D17B001263B9801A1964202020202020202020202020204B6579735F537472
:2039EE00617475739039D97D007C017F197E001262D17B001263B9801B1A482F6820202068
:203A0E002020202020202020416C61726D204F46462F4F4E903A087D007C017F1A7E0012EF
:203A2E0062D17B001263B980201F69206E2020202020202020202020496E70757420766F71
:203A4E006C7461676520476574903A387D007C017F1F7E001262D17B001263B9802F2E4BDD
:203A6E002F6B20202020202020202020204B6579204C4F434B20287374617274205761740A
:203A8E006368646F67292F554E4C4F434B903A6D7D007C017F2E7E001262D17B001263B9A5
:203AAE008026254C206E2F6C206E202020202020204C69737420414443732C444143732FBD
:203ACE00766F6C7461676573903AB17D007C017F257E001262D17B001263B9801B1A4D20CC
:203AEE006E2F6D2020202020202020204D6F6465205365742F476574903AEC7D007C017F3F
:203B0E001A7E001262D17B001263B98016156E206E20202020202020202020204441432022
:203B2E00676574903B1C7D007C017F157E001262D17B001263B98025244F206E2C6461635C
:203B4E002F6F206E2020204441435F4F7665725F4C696D6974205365742F476574903B47FD
:203B6E007D007C017F247E001262D17B001263B98039385020612C732C6C2C722C692F7063
:203B8E0020537061726B20506172616D7328416D706C2C53686F72742C4C656E2C526563F3
:203BAE006F7629205365742F476574903B817D007C017F387E001262D17B001263B980263F
:203BCE002551206E2F71206E20202020202020537061726B20436F756E74657220436C6590
:203BEE0061722F476574903BCF7D007C017F257E001262D17B001263B980292852206E2C14
:203C0E00612C622F72206E2020205265736973746F7273283130204F686D73292053657495
:203C2E002F476574903C0A7D007C017F287E001262D17B001263B9801C1B7320202020207A
:203C4E0020202020202020205374617475732028303D6F6B29903C487D007C017F1B7E00F4
:203C6E001262D17B001263B980272654206E2F74202020202020202020526567756C617402
:203C8E00696F6E2044656C6179205365742F476574903C797D007C017F267E001262D17B04
:203CAE00001263B980222156206E2C762F76206E2020202020412D4220766F6C74616765EA
:203CCE00205365742F476574903CB57D007C017F217E001262D17B001263B980292857206C
:203CEE006E2C762F77206E2020202020526567756C6174696F6E2077696E646F777320531A
:203D0E0065742F476574903CEC7D007C017F287E001262D17B001263B9802322582F7820C4
:203D2E0020202020202020202020537061726B204D6F6E69746F72204F4E2F4F4646903D98
:203D4E002A7D007C017F227E001262D17B001263B98022215E20636F646520202020202088
:203D6E0020205361766520736574757020696E20666C617368903D627D007C017F217E00A9
:203D8E001262D17B001263B98021202020202020202020202020202020416C6C20566F6C3C
:203DAE00746167657320696E205621903D997D007C017F207E001262D17B001263B9803533
:203DCE00342D2D2D2D2D2D2D2D2D2D2D2D2D2D2D2D2D2D2D2D2D2D2D2D2D2D2D2D2D2D2D2E
:203DEE002D2D2D2D2D2D2D2D2D2D2D2D2D2D2D2D2D2D2D2D2D903DCF7D007C017F347E003D
:203E0E001262D17B001263B922800100903E197C8C7D8275070A7506001264D9740190823E
:203E2E0099F0908299E0D394084003023E72309803023E4480F8C298E599640D6003023E49
:203E4E005022908299E090828CF0908299E090828C2582F58250020583E599F0908299E0AF
:203E6E0004F080BE22123E1790828CC082C083908297D005D004126240EC908296F09082BA
:203E8E0097E0FAA3E0FBEA90828AF0A3EBF02290829CE0FCA3E0FD8C828D83C082C08374EE
:203EAE000090816AF0A37400F0740890816CF0A37400F01204CED083D082C082C083908173
:203ECE006EE0D083D082F090829CE0FCA3E0FD8C828D83E06003023F0890829AE0FCA3E032
:203EEE00FD8C828D837401F090829CE0FCA3E0FD8C828D837408F0023F2A90829AE0FCA30A
:203F0E00E0FD8C828D83C082C08390829CE0FCA3E0FD8C828D83E0D083D082F02290829EA4
:203F2E00E0908180F07401908181F01205CF741F908183F0A37400F0741F908185F0A374E7
:203F4E0000F012077E740D908199F0740090819AF0A37400F0120AA1740D908195F0740251
:203F6E00908196F01209CD74FB90F7D0F0740E908199F0908023E0FAA3E0FBEA90819AF0D2
:203F8E00A3EBF0120AA1740E908195F07402908196F01209CD74FB90F7E0F0C20B2220985E
:203FAE0003024E55E59964216003024019C298123E7390828AE0FAA3E0FBEA90829FF0A34B
:203FCE00EBF0908001E0FCA3E0FD90829FE0FEA3E0B50507EEB50403023FED740080027476
:203FEE0001FE90829FE0FAA3E0B40006BA000302400474008002740113EE72E040030240A6
:20400E0014D208024016C208024E55200803024E537B001262CCEA9082ADF09082ADE0FE1E
:20402E00EE643F600302403C123653024077EE645E600302407A74D090816AF0A3748AF09D
:20404E00743090816CF0A37475F01204CE90816EE0FEA3E0B40406BEE00302406E0240743C
:20406E0012345D0240771233A40240A9EE642360030240AC740090816AF0A37400F07430B2
:20408E0090816CF0A37475F01204CE90816EE0FAA3E0FBEA908001F0A3EBF0024105EE646B
:2040AE00266003024108740090816AF0A37400F0741F90816CF0A37400F01204CE90816ECE
:2040CE00E0FAA3E0FBEA908023F0A3EBF0740090816AF0A37400F0740690816CF0A374000B
:2040EE00F01204CE90816EE0908025F0908025E090829EF0123F2B0241E9EE644160030205
:20410E0041EC74AF90829AF0A37482F074B090829CF0A37482F0123E9D74F090816AF0A372
:20412E0074D8F0740090816CF0A37400F01204CE90816EE0FAA3E0FBEA90829FF0A3EBF089
:20414E009082AFE09082AEF09082B0E0FE9082AEE0D39E40030241E9125D3A0000C842121B
:20416E005D3A00004842125C2390829FE0FAA3E0FB7401125AEF125CA19082AEE075F00290
:20418E00A490809F2582F58250020583E0FAA3E0FB7401125AEF125C23125ABC125ACEEAC1
:2041AE0090829FF0A3EBF09082AEE075F002A49080112582F58250020583C082C083908277
:2041CE009FE0FAA3E0FBEAD083D082F0A3EBF09082AEE004F0600302415600024252EE6465
:2041EE0061600302425574AF90829AF0A37482F074B090829CF0A37482F0123E9D9082AF13
:20420E00E09082AEF09082B0E0FE9082AEE0D39E40030242529082AEE075F002A49080AF0C
:20422E002582F582500205837E007F01E0FAA3E0FB12632B7B001263B99082AEE004F060E5
:20424E000380C200024336EE6442600302433974AF90829AF0A37482F074B090829CF0A36E
:20426E007482F0123E9D74F090816AF0A374D8F0740090816CF0A37400F01204CE90816E64
:20428E00E0FAA3E0FBEA90829FF0A3EBF09082AFE09082AEF09082B0E0FE9082AEE0D39EAD
:2042AE004003024336125D3A0000C842125D3A00004842125C2390829FE0FAA3E0FB74013D
:2042CE00125AEF125CA19082AEE075F002A490808F2582F58250020583E0FAA3E0FB740157
:2042EE00125AEF125C23125ABC125ACEEA90829FF0A3EBF09082AEE075F002A49080012578
:20430E0082F58250020583C082C08390829FE0FAA3E0FBEAD083D082F0A3EBF09082AEE091
:20432E0004F060030242A30002439FEE646260030243A274AF90829AF0A37482F074B09053
:20434E00829CF0A37482F0123E9D9082AFE09082AEF09082B0E0FE9082AEE0D39E40030284
:20436E00439F9082AEE075F002A49080BF2582F582500205837E007F01E0FAA3E0FB126310
:20438E002B7B001263B99082AEE004F0600380C2000243CCEE644360030243CF740190815F
:2043AE006AF0A37400F0740890816CF0A37400F01204CE90816EE0908248F01221EE0243AB
:2043CE00EAEE646360030243ED7E007F01908027E0FA7B0012632B7B001263B9024440EE54
:2043EE00644460030244437B00126268EA90829FF0A3EBF07B007C099082A31262067B0011
:20440E001263B9C20D90829FE090812CF09082A37C2D7D8175070A7506001264B3120180BA
:20442E0090829FE0FEA3E0B40006BE0003024440D20D024461EE6464600302446412031CE1
:20444E007E007F0190815EE0FA7B0012632B7B001263B9024471EE64486003024474C21102
:20446E00121E9A024481EE64686003024484D211121E9A0244EAEE646960030244ED74AF65
:20448E0090829AF0A37482F074B090829CF0A37482F0123E9D9082AFE09082AEF09082B09E
:2044AE00E0FE9082AEE0D39E40030244EA9082AEE075F002A49080CF2582F582500205830A
:2044CE007E007F01E0FAA3E0FB12632B7B001263B99082AEE004F0600380C2000244FAEEC8
:2044EE00644B60030244FD1200D1D20E024507EE646B600302450AC20E0245A9EE644C6019
:20450E00030245AC74AF90829AF0A37482F074B090829CF0A37482F0123E9D9082AFE090E6
:20452E0082AEF09082B0E0FE9082AEE0D39E40030245A99082AEE075F002A490809F258268
:20454E00F582500205837E007F06E0FAA3E0FB12632B9082AEE075F002A490808F2582F51B
:20456E0082500205837E007F06E0FAA3E0FB12632B9082AEE09080702582F58250020583BE
:20458E007E007F06E0FA7B0012632B7B001263B99082AEE004F0600380890002468FEE6443
:2045AE006C600302469274AF90829AF0A37482F074B090829CF0A37482F0123E9D9082AF03
:2045CE00E09082AEF09082B0E0FE9082AEE0D39E400302468F9082AEE075F002A49080CFE8
:2045EE002582F582500205837E007F06E0FAA3E0FB12632B9082AEE075F002A49080AF252B
:20460E0082F582500205837E007F06E0FAA3E0FB12632B9082AEE075F002A49080BF25829D
:20462E00F582500205837E007F06E0FAA3E0FB12632B9082AEE075F002A49080DF2582F5EA
:20464E0082500205837E007F06E0FAA3E0FB12632B9082AEE075F002A490807F2582F5829D
:20466E00500205837E007F06E0FAA3E0FB12632B7B001263B99082AEE004F060030245D39D
:20468E00000246C1EE644D60030246C4740090816AF0A37400F0740490816CF0A37400F023
:2046AE001204CE90816EE09082AEF09082AEE0908000F00246DFEE646D60030246E27E0068
:2046CE007F01908000E0FA7B0012632B7B001263B9024743EE646E600302474674AF90822B
:2046EE009AF0A37482F074B090829CF0A37482F0123E9D9082AFE09082AEF09082B0E0FE70
:20470E009082AEE0D39E40030247439082AEE09080702582F582500205837E007F01E0FABB
:20472E007B0012632B7B001263B99082AEE004F0600380C700024797EE644F600302479AA2
:20474E0074AF90829AF0A37482F074B090829CF0A37482F0123E9D9082AFE0908286F09012
:20476E0082B0E0908287F0743290816AF0A37400F074F290816CF0A37400F01204CE9081A9
:20478E006EE0908288F01235C70247FBEE646F60030247FE74AF90829AF0A37482F074B00A
:2047AE0090829CF0A37482F0123E9D9082AFE09082AEF09082B0E0FE9082AEE0D39E400392
:2047CE000247FB9082AEE09080782582F582500205837E007F01E0FA7B0012632B7B0012E7
:2047EE0063B99082AEE004F0600380C7000248A2EE645060030248A574D090816AF0A374AB
:20480E008AF0743090816CF0A37475F01204CE90816EE0FAA3E0FBEA90806FF0A3EBF0747D
:20482E00D090816AF0A3748AF0740090816CF0A37400F01204CE90816EE0FAA3E0FBEA9081
:20484E00806DF0A3EBF0740090816AF0A37400F0743090816CF0A37475F01204CE90816E19
:20486E00E0FAA3E0FBEA90804BF0A3EBF0740090816AF0A37400F0743090816CF0A374759C
:20488E00F01204CE90816EE0FAA3E0FBEA908049F0A3EBF0024918EE6470600302491B7E42
:2048AE00007F0190806FE0FAA3E0FB12632B7420FA7C017D007E047F011262D17E007F0126
:2048CE0090806DE0FAA3E0FB12632B7420FA7C017D007E047F011262D17E007F0190804B2D
:2048EE00E0FAA3E0FB1263217420FA7C017D007E047F011262D17E007F01908049E0FAA319
:20490E00E0FB1263217B001263B9024977EE6451600302497A74AF90829AF0A37482F07426
:20492E00B090829CF0A37482F0123E9D9082AFE09082AEF09082B0E0FE9082AEE0D39E4063
:20494E00030249779082AEE075F002A49080372582F582500205837400F0A37400F090821D
:20496E00AEE004F0600380CC000249E0EE647160030249E374AF90829AF0A37482F074B00D
:20498E0090829CF0A37482F0123E9D9082AFE09082AEF09082B0E0FE9082AEE0D39E4003B0
:2049AE000249E09082AEE075F002A49080372582F582500205837E007F01E0FAA3E0FB126C
:2049CE0063217B001263B99082AEE004F0600380C200024AC3EE64526003024AC674AF9088
:2049EE00829AF0A37482F074B090829CF0A37482F0123E9D740090816AF0A37400F0743052
:204A0E0090816CF0A37475F01204CE90816EE0FAA3E0FBEA90829FF0A3EBF0740090816AEC
:204A2E00F0A37400F0743090816CF0A37475F01204CE90816EE0FAA3E0FBEA9082A1F0A3F9
:204A4E00EBF09082AFE09082AEF09082B0E0FE9082AEE0D39E4003024AC39082AEE075F014
:204A6E0002A49080112582F58250020583C082C08390829FE0FAA3E0FBEAD083D082F0A3B9
:204A8E00EBF09082AEE075F002A49080012582F58250020583C082C0839082A1E0FAA3E0E4
:204AAE00FBEAD083D082F0A3EBF09082AEE004F06003809600024B59EE64726003024B5C6D
:204ACE0074AF90829AF0A37482F074B090829CF0A37482F0123E9D9082AFE09082AEF09067
:204AEE0082B0E0FE9082AEE0D39E4003024B599082AEE075F002A49080112582F582500262
:204B0E0005837E007F07E0FAA3E0FB12632B7420FA7C017D007E047F011262D19082AEE094
:204B2E0075F002A49080012582F582500205837E007F07E0FAA3E0FB12632B7B001263B9AE
:204B4E009082AEE004F06003809500024B85EE64736003024B887E007F01908030E0FA7BD9
:204B6E000012632B7E007F01908123E0FA7B0012632B7B001263B9024BAFEE6454600302B0
:204B8E004BB2740090816AF0A37400F074FF90816CF0A37400F01204CE90816EE0908121C8
:204BAE00F0024BCDEE64746003024BD07E007F03908121E0FA7B0012632B7B001263B902C5
:204BCE004C54EE64566003024C5774AF90829AF0A37482F074B090829CF0A37482F0123E94
:204BEE009D74F090816AF0A374D8F0740090816CF0A37400F01204CE90816EE0FAA3E0FBB9
:204C0E00EA90829FF0A3EBF09082AFE09082AEF09082B0E0FE9082AEE0D39E4003024C5496
:204C2E009082AEE0908238F090829FE0FAA3E0FBEA908239F0A3EBF0121BBA9082AEE00455
:204C4E00F0600380CB00024CBDEE64766003024CC074AF90829AF0A37482F074B090829C4A
:204C6E00F0A37482F0123E9D9082AFE09082AEF09082B0E0FE9082AEE0D39E4003024CBD70
:204C8E009082AEE075F002A49080DF2582F582500205837E007F01E0FAA3E0FB12632B7B03
:204CAE00001263B99082AEE004F0600380C200024D44EE64576003024D4774AF90829AF08B
:204CCE00A37482F074B090829CF0A37482F0123E9D740090816AF0A37400F074E890816C46
:204CEE00F0A37403F01204CE90816EE0FAA3E0FBEA90829FF0A3EBF09082AFE09082AEF097
:204D0E009082B0E0FE9082AEE0D39E4003024D449082AEE090823CF090829FE0FAA3E0FB17
:204D2E00EA90823DF0A3EBF0121C859082AEE004F0600380CB00024DADEE64776003024D52
:204D4E00B074AF90829AF0A37482F074B090829CF0A37482F0123E9D9082AFE09082AEF0C4
:204D6E009082B0E0FE9082AEE0D39E4003024DAD9082AEE075F002A49080FF2582F582500D
:204D8E000205837E007F01E0FAA3E0FB12632B7B001263B99082AEE004F0600380C20002A1
:204DAE004DBDEE64586003024DC0D212122BCF024DCDEE64786003024DD0C212122BCF0285
:204DCE004E27EE642A6003024E2A7B001262CCEA9082ADF09082ADE0FEEE64436003024DBF
:204DEE00F4D20B024DFEEE64636003024E01C20B024E277407FA7C017D007E047F011262F5
:204E0E00D1800302203F904E127D007C017F027E001262D17B001263B9024E507407FA7C67
:204E2E00017D007E047F011262D1800302203F904E3B7D007C017F027E001262D17B0012D7
:204E4E0063B9024E55C29822908001E0FAA3E0FB9082B17F07E4126147908023E0FAA3E027
:204E6E00FB9082BB7F05E41261477423FB7A011261EA7802E41261669082B1740112616688
:204E8E007C457D8175070A7506001264B380040343414E1261EA904E9D7402126166908289
:204EAE00BB74011261667C4F7D8175070A7506001264B374D0908159F0A37407F01202A583
:204ECE00221200D49082C5E09081A1F0120C589081A2125FC77401125F63EA9082C6F0A364
:204EEE00EBF09082C5E09081AFF074D09081B0F0A37482F09082C8AA82AB83EA9081B2F013
:204F0E00A3EBF0120F23200B03024F449082C6E0FAA3E0FBEA90822AF0A3EBF09082D0E078
:204F2E0090822CF09082C8AA82AB83EA90822DF0A3EBF01219D89082C6E0FAA3E0FBEA90BD
:204F4E0081C8F0A3EBF01212959081CAE0FEEE6003024FB774019081CFF074009081D0F037
:204F6E00A37400F074039081D2F0908028E09081D3F0A20974003354019081D4F090812336
:204F8E00E09081D5F074009081D6F074009081D7F074009081D8F074009081D9F074009017
:204FAE0081DAF01212D0024FCDEE64016003024FD09082C8E0640124FFB39211121E9A024B
:204FCE005023EE6402600302502674019081CFF074029081D0F0A37400F074019081D2F046
:204FEE00908030E09081D3F074009081D4F074009081D5F074009081D6F074009081D7F085
:20500E0074009081D8F074009081D9F074009081DAF01212D0025039EE6404600302503CD2
:20502E009082C8E0908249F0122231025098EE6405600302509B74C89081F0F0A37482F0B1
:20504E0074D19081F2F0A37482F012139C9082C8E09082D0F09082D1E0FE9082D0E0D39E40
:20506E0040030250989082D0E075F002A49080372582F582500205837400F0A37400F090EE
:20508E0082D0E004F0600380CC000250FCEE640660030250FF74019081CFF074069081D033
:2050AE00F0A37400F074089081D2F0908070E09081D3F090806FE09081D4F090806EE09046
:2050CE0081D5F090806DE09081D6F090804CE09081D7F090804BE09081D8F090804AE09056
:2050EE0081D9F0908049E09081DAF01212D0025193EE640760030251969082C8E0908230C9
:20510E00F09082C9E0908231F0121A69908232E0FAA3E0FBEA90806FF0A3EBF09082CAE0DF
:20512E00908230F09082CBE0908231F0121A69908232E0FAA3E0FBEA90806DF0A3EBF090A9
:20514E0082CCE0908230F09082CDE0908231F0121A69908232E0FAA3E0FBEA90804BF0A3E6
:20516E00EBF09082CEE0908230F09082CFE0908231F0121A69908232E0FAA3E0FBEA908035
:20518E0049F0A3EBF00251A9EE640960030251AC9082C8E0908209F01218A602522CEE642A
:2051AE0020600302522F74C89081F0F0A37482F074D19081F2F0A37482F012139C9082C9C8
:2051CE00E0FAA3E0FBEA90820CF0A3EBF012193A90820EE0FAA3E0FBEA9082D2F0A3EBF0DA
:2051EE009082C8E09082D0F09082D1E0FE9082D0E0D39E400302522C9082D0E0908238F062
:20520E009082D2E0FAA3E0FBEA908239F0A3EBF0121BBA9082D0E004F0600380CB00025202
:20522E0042EE642260030252459082C8E09081F4F01213F2025258EE6424600302525B9024
:20524E0082C8E09081F7F01214A20252DBEE642560030252DE74C89081F0F0A37482F074F1
:20526E00D19081F2F0A37482F012139C9082C9E0FAA3E0FBEA90820CF0A3EBF012193A9074
:20528E00820EE0FAA3E0FBEA9082D2F0A3EBF09082C8E09082D0F09082D1E0FE9082D0E0CD
:2052AE00D39E40030252DB9082D0E090823CF09082D2E0FAA3E0FBEA90823DF0A3EBF01208
:2052CE001C859082D0E004F0600380CB000252F1EE642760030252F49082C8E09081FAF09D
:2052EE00121552025307EE6429600302530A9082C8E09081FDF012160202531DEE642B605D
:20530E00030253209082C8E0908200F01216B2025333EE642D60030253369082C8E09082B0
:20532E0003F0121762025370EE642E600302537374C89081F0F0A37482F074D19081F2F083
:20534E00A37482F012139C9082C8E0908286F09082D1E0908287F09082C9E0908288F01210
:20536E0035C7025386EE643060030253899082C8E0908206F0121812025399EE64316003B3
:20538E0002539C9082C8E0908121F00253EFEE643260030253F274019081CFF074329081C4
:2053AE00D0F0A37400F074019081D2F0908121E09081D3F074009081D4F074009081D5F057
:2053CE0074009081D6F074009081D7F074009081D8F074009081D9F074009081DAF012121A
:2053EE00D0025429EE6433600302542C9082C8E0908162F0A3740000F07401908164F0A345
:20540E007400F07408908166F0A37400F0120459908168E0908248F01221EE02547FEE64D6
:20542E0034600302548274019081CFF074349081D0F0A37400F074019081D2F0908027E0CB
:20544E009081D3F074009081D4F074009081D5F074009081D6F074009081D7F074009081BB
:20546E00D8F074009081D9F074009081DAF01212D00254CFEE643560030254D2C20D9082AD
:20548E00C8E090812CF09082D0E0C39401908212F09082C9AA82AB83EA908213F0A3EBF049
:2054AE0012195B9082157C2D7D8175070A7506001264B31201809082C8E070030254CFD2A9
:2054CE000D025528EE6436600302552B74019081CFF074369081D0F0A37400F07401908178
:2054EE00D2F012031C90815EE09081D3F074009081D4F074009081D5F074009081D6F07436
:20550E00009081D7F074009081D8F074009081D9F074009081DAF01212D0025575EE643772
:20552E0060030255789082C8E0FEEE6003025543C20E02554DEE64016003025550D20E02D5
:20554E00555BEE6402600302555E1200D1025572EE640360030255751200D1D2BE800302F9
:20556E00557280F90255750255B4EE643860030255B79082C8E0908162F0A3740000F07473
:20558E0000908164F0A37400F07403908166F0A37400F0120459908168E09082D0F0908200
:2055AE00D0E0908000F002560AEE6439600302560D74019081CFF074399081D0F0A374009E
:2055CE00F074019081D2F0908000E09081D3F074009081D4F074009081D5F074009081D6D3
:2055EE00F074009081D7F074009081D8F074009081D9F074009081DAF01212D0025666EED7
:20560E00643A600302566974019081CFF0743A9081D0F0A37400F074069081D2F07401909D
:20562E0081D3F074589081D4F0908002E09081D5F0908001E09081D6F0908024E09081D7EB
:20564E00F0908023E09081D8F074009081D9F074009081DAF01212D0025710EE643B600376
:20566E000257139082C8E0908230F09082C9E0908231F0121A69908232E0FEA3E0B40106E1
:20568E00BE5303025698740080027401FEC0069082CAE0908230F09082CBE0908231F012D9
:2056AE001A69D006908001E0FCA3E0FD908232E0FAA3E0B50507EAB504030256CF740080F3
:2056CE0002740113EE82E040030257109082CCE0908230F09082CDE0908231F0121A69902F
:2056EE008232E0FAA3E0FBEA908023F0A3EBF09082CEE0908025F0908025E090829EF01259
:20570E003F2B02573EEE643C600302574174019081E3F0743C9081E4F0A37400F09000B7B3
:20572E007CE67D8175070A7506001264D912135602576CEE643D600302576F74019081E348
:20574E00F0743D9081E4F0A37400F09000C87CE67D8175070A7506001264D91213560257D2
:20576E00C8EE643E60030257CB74019081CFF0743E9081D0F0A37400F074019081D2F09095
:20578E00817FE09081D3F074009081D4F074009081D5F074009081D6F074009081D7F074A9
:2057AE00009081D8F074009081D9F074009081DAF01212D0740090817FF00257CB9082C582
:2057CE00E075F010A490F7002582F5825002058374FDF022C0D075D000C0E0C0F0C082C099
:2057EE00839082D412652B90F702E0C394029082C5F0124ECF9082D412654ED083D082D0B8
:20580E00F0D0E0D0D0327400908283F0123364758680E5A9FEEE54406440600302583C90B0
:20582E008123E02401908123F0D20C0258447400908123F0C20C7B00126692758DF575902A
:20584E000B1203071202E8121C40121CC812215D9000B77C457D8175070A7506001264D9CD
:20586E009000C87C4F7D8175070A7506001264D974D0908159F0A37407F01202A51234F905
:20588E00124E56908025E090829EF0123F2B800908202020202043682D90589E7C457D81C5
:2058AE0075070A7506001264D98009084D6F64652043682B9058B97C4F7D8175070A750613
:2058CE00001264D974D0908159F0A37407F01202A57401908248F01221EE7402908000F0B0
:2058EE00D2087400908121F0908121E0908122F0C211121E9AC212122BCF121F10200C0308
:20590E0002595C74019081CFF074009081D0F0A37400F074029081D2F074009081D3F09010
:20592E008123E09081D4F074009081D5F074009081D6F074009081D7F074009081D8F0745E
:20594E00009081D9F074009081DAF01212D01200D4121F101222E11225AC1200D4122BD406
:20596E00123FAC1227DF80E680FE88528B518C537524017A007B00125AEFC214752500121F
:20598E006581C213EAC3942D700BD2137524021265810259AFEAC3942B70067524021265DF
:2059AE0081EAC39430B333FBEAC394396001B3B3EB82E033FBEAC3942EC37001D3EB72E097
:2059CE004003025A0A2014030259DB0525EAC3942E60030259E9D214025A05C0027A0A7B5B
:2059EE0000125AEF125C23D0E0C39430FA7B00125AEF125BAF052412658180A5201403020B
:205A0E005A2BE525C394006001B34003025A2B7A0A7B00125AEF125CA1152580E520130376
:205A2E00025A34125ABC22ECC0E0E604FCF526087B05125978D001125DB912626122C08353
:205A4E00C0828C828D83E0A304FCF5267B06125978D082D083125DEC12626122E54DA2E724
:205A6E009216D2E7F54DE548A2E79217D2E7F548E54EC395494011E54E6549601CC378451E
:205A8E001260220549025A85E549654E600BC3784A126022054E025A9622E6C397F6080922
:205AAE00E697F60809E697F60809E697F622E54E6006E54DB2E7F54D22E54DC2E7F54D2234
:205ACE00E54D20E70E125D3A0000003F125BAF125B5422125D3A0000003F125BAC125B54C8
:205AEE0022602012609E8B4D8A4C754B00754A00EBA2E792165005784A126074754E8E123D
:205B0E0060352212609E8B4D8A4C754B00754A00C21680E8E54DA2E79216D2E7F54DC3E53D
:205B2E004E949EF54E500FE54E601A784AC3126022054E025B35E54E600B784AC3126012E3
:205B4E00154E025B4422E54E6018125B22AA4AAB4B30160AEAF42401FAEBF43400FB126020
:205B6E008C227A007B0012608C22E54E6023125B2230161CE54AF42401F54AE54BF43400CE
:205B8E00F54BE54CF43400F54CE54DF43400F54D22754A00754B00754C00754D0022125ACF
:205BAE00BCE54E603CE5496035125A6AA21692E7A21765D020E7137945784A1260615007D0
:205BCE00784A126022054E025BE87945784A125AA85007784A126074B21612603522125D36
:205BEE00FD12608C22E687F0A4FCADF008E687F0A42DFDE435F0FEE433FF1809E687F0A46E
:205C0E002DFDE5F03EFEE43FFF08E687F0A42EFEEF35F0FF22E54E7003025BECE54970031F
:205C2E00025BEFE548A2E79216D2E7F548E54DA2E7D2E7F54D5002B216784C7945125BF304
:205C4E00EEFAEFFB784A7947125BF3EE2AFAEF3BFB9217784C7947125BF3EC2AF54AED3B41
:205C6E00F54BE43EC0D0A2173400F54CE4D0D03FF54DE549254E2482F54E126035227549E0
:205C8E007F7548FF7547FF7546FF7545FF12608CD2D222E54E60E7E5497003025BEFE54835
:205CAE00A2E79216D2E7F548E54DA2E7D2E7F54D5002B216C37845126022C3784A126022B2
:205CCE00AC45AD46AE47AF4875450075460075470075480075F02015F0E5F06035C3EC95C0
:205CEE004AED954BEE954CEF954D4011C3EC954AFCED954BFDEE954CFEEF954DFFB378452D
:205D0E00126012E5D0541804040404F8126012025CE550057845126022E549C2D7954E248D
:205D2E0080F54912608C126035C2D22212609ED083D082784A7600087904740093F608A322
:205D4E0019E970F6C082C083125D5E2212609E22E54DA2E7E54E33F54EE54D92E7F54D22B4
:205D6E00E54DA2E7E54E13F54EE54D92E7F54D22E8C0E012609ED0E0F8794A7700097F04BC
:205D8E0012649E125D5E22E54A30E71E784AE62401F608E63400F608E63400F608E6340079
:205DAE00F65007784A126022054E22125D95125D6E784B7F0412649E12608C2212609E79D9
:205DCE004A7700097F041264AC125D5E2212609E794A7700097F041264D0125D5E22125DDD
:205DEE0095125D6E784B7F041264A512608C22784A79457A05E6FBE7F6EBF70809DAF62200
:205E0E00E548A2E7B3E54913F549E54892E7F548E54DA2E7B3E54E13F54EE54D92E7F54DC5
:205E2E00E54E20E70DE54920E7087849794E7F058006784E79497F05C3E79670041819DF6E
:205E4E00F7FA13FB12611D12611DEB33EA22125D5A125C2322E54D3392165003125E9DE51D
:205E6E00483392175019C374009545F54574009546F54674009547F54774009548F5482276
:205E8E00A21633F8A217336830E0F4125E9D22C37400954AF54A7400954BF54B7400954C4C
:205EAE00F54C7400954DF54D22E54D30E703125E9D22784A7945126061227845794AC37A2C
:205ECE0004E697F70809DAF9227845794A7A04E657F70809DAF9227845794A7A04E647F7DC
:205EEE000809DAF922E54A60097845126022154A80F312608C22E54A6009784512601215C5
:205F0E004A80F312608C22125E631260B0C3784A126022125E8E22125E631260D912608C4C
:205F2E00125E8E22125E631260D98C458D468E478F48784512602212608C2212609ED083F1
:205F4E00D082784A7904740093F608A319E970F6C082C08322600814602714602C8019129D
:205F6E00609E8A4A8B4BEB30E707754CFF754DFF22754C00754D002212609E8A4A8B4B80E0
:205F8E00F0AA4AAB4B12608C22754E9EE54DA2E792165005784A12607412603522E8C0E0E7
:205FAE0012609ED0E0F8794A7F0412649E22784A7F0412649E12608C2212609E794A7F04D0
:205FCE001264AC2212609E794A7F041264D022784A7F041264A512608C22E54D6480F8C360
:205FEE00E5486480987010E547954C700AE546954B7004E545954AFBACD012611D12611DC4
:20600E008CD0EB22E633F608E633F608E633F608E633F622080808E613F618E613F618E687
:20602E0013F618E613F6227920E54D20E71C784AC3126012154E19E970EF754E00754D00E0
:20604E00754C00754B00754A0022E54DA21692E7F54D22E627F60809E637F60809E637F6BE
:20606E000809E637F622E6F42401F608E6F43400F608E6F43400F608E6F43400F622784ECB
:20608E00794975F005E7F6181915F0E5F070F6227845794A75F005E7F6080915F0E5F07034
:2060AE00F6227C007D007E007F0075F02115F0E5F06017784A12602230D70778047945123D
:2060CE00606178041260220260BB227C007D007E007F0075F021C3EC954AED954BEE954CFC
:2060EE00EF954D4011C3EC954AFCED954BFDEE954CFEEF954DFFB37845126012E5D054186A
:20610E0004040404F812601215F0E5F070C82212608C22D03BD03CC045C046C047C048C0A0
:20612E0049C03CC03B22D03BD03CD049D048D047D046D045C03CC03B22C082C083A37E06A0
:20614E007553006005126321800312632BE553D083D082F0220261C960FB14603174009329
:20616E006025F53FA374009385823B85833C0540853D82853E83F0A385823D85833E853B7C
:20618E0082853C83D53FDD9082F3E540F022E06023F53FA3E085823B85833C0540853D82D5
:2061AE00853E83F0A385823D85833E853B82853C83D53FDF9082F3E540F022E66011F53F2E
:2061CE00853D82853E83054008E6F0A3D53FF785823D85833E9082F3E540F02285823B85C9
:2061EE00833C9082F37400F0F540A385823D85833E853B82853C8322AD82AE837F008B51A4
:20620E00126581EA640D6006A30FEAF0DCF28D828E83EFF022ECC0E07B05E608885204F56F
:20622E0053F526126268D0E0F8EAF608EBF612626122C082C0838C828D837B06E0A304F5FE
:20624E0053F526126268D083D082EAF0A3EBF012626122C3E5269553FC228B51752900752F
:20626E002A001265818A2BC200E52B642D7007D2001265818A2BE52BC39430B333FAE52B59
:20628E00C394396001B3B3EA82E0501F7C0A7D00AA29AB2A1263CEE52BC394302AF529EB26
:2062AE003400F52A1265818A2B80CB30000BAA29AB2A12646D8A298B2AAA29AB2A228B51B1
:2062CE000265818D51ECC39F400E600CFCEAFD7A2012660BDCF9EDFAEF600FEE602A1460DC
:2062EE001514601B14600412660B22EAFA12660BEBFA12660B22E6FA12660B08DFF822E09A
:20630E00A3FA12660BDFF822740093A3FA12660BDFF6228E518F398A2C8B2D80218E518F14
:20632E00398A2C8B2DEB30E715D215E53960021539AA2CAB2D12646D8A2C8B2D8002C21584
:20634E00753A04E53A242FF87C0A7D00AA2CAB2D126400EA2430F67C0A7D00AA2CAB2D12F4
:20636E0063F08A2C8B2DE53960021539153AE52C452D70CF752E01E539C3952E400B7A2042
:20638E0012660B052EE52E70EE3015057A2D12660B053A7404C3953A4010E53A242FF8E66B
:2063AE00FA12660B053AE53A70E9228B517A0D12660B7A0A12660B2222EA2CFAEB3DFB22F3
:2063CE00EEC0E0EFC0E0EA8CF0A4FEAFF0EA8DF0A42FFFEB8CF0A42FFBEEFAD0E0FFD0E036
:2063EE00FE22EEC0E0EFC0E0126424D0E0FFD0E0FE22BB000ABD0007EA8CF084AAF022EE1C
:20640E00C0E0EFC0E0126424C3EF13FBEE13FAD0E0FFD0E0FE22BB000DBD000AEA8CF084F2
:20642E00FAAEF07F0022E8C0E0E9C0E075F0117E007F00EEF8EFF9C2D7EE9CFEEF9DFFB364
:20644E004004E8FEE9FFEA33FAEB33FBEE33FEEF33FF15F0E5F070DBD0E0F9D0E0F822EB29
:20646E00F4FBEAF404FA70010B22EC6009C3EA33FAEB33FBDCF722EC6009C3EB13FBEA135A
:20648E00FADCF722FDEC6006C3ED33FDDCFAED22E6F70809DFFA22E6F008A3DFFA22E0F7AF
:2064AE0009A3DFFA22EF60010EE0A3AA82AB838C828D83F0A3AC82AD838A828B83DFEADE1C
:2064CE00E822740093F709A3DFF822EF60010E740093A3AA82AB838C828D83F0A3AC82AD13
:2064EE00838A828B83DFE8DEE622E6FCE0FDEC600EED601008A31C1DC3E09660F1B322ED9E
:20650E006003D322ECC322EA9CEDF5F06480FDEB64809DADF022E608F0A3D9FA22E8F0A3EF
:20652E00E9F0A378027906126524783B7914126524A21633A21733F022E0A3F608D9FA2203
:20654E00E0C0E0A3E0C0E0A378027906126547783B7914126547E0139217139216D001D03A
:20656E0000228A828B8374007390834485824F85835022E55160491414605514607D1460A2
:20658E007B14602F14601F14601030C0FDC2C0E5C1FA940D600312660B22E59B30E0FBC2B3
:2065AE00E0F59BAA9C221553E5536004E0A3FA227A0D221553E55360F7A852E60552FA225F
:2065CE003098FDC298E599FA940D600312660B22D2AF20B2FBC2AF7DBADDFE20B2F27A0757
:2065EE00C312660412660413A2B2DAF513C313126604FAD2AF227DBADDFE222222E551608C
:20660E003914603F14605214607814607614602114601814600930C1FDEAF5C1C2C122E52E
:20662E009B30E1FBC2E1F59B8A9C22EAF0A3055322EAA852F605520553223099FDEAF5994A
:20664E00C29922C083C082906100E0E020E7FB906200EAF0D082D08322C2AFC2B512668BF9
:20666E0012668B7C07EA13FA92B512668B12668BDCF3D2B512668B12668BD2AF227DBADD2F
:20668E00FE222222EB602AB40708759DDC759B93801EB4081BE589540F2420F589C2C7D25C
:2066AE00C6758DFAD28EE5874480F587D2C4D2C122E589540F2420F589C29FD29E758DFA53
:2066CE00D28EE5874480F587D29CD299C20122755480D000D001855481C001C00022755432
:0F66EE0055D000D001855481C001C000D21822C0
:00000001FF
